:100000000C9418050C945F050C9454080C945F052F
:100010000C945F050C945F050C945F050C945F05D0
:100020000C945F050C945F050C94330E0C94050F33
:100030000C945E1C0C945F050C945F050C945F059A
:100040000C945F050C945F050C945F050C945F05A0
:100050000C945F050C94D21C0C945F050C945F0506
:100060000C945F050C945F050C945F050C945F0580
:100070000C945F050C945F050C945F050C945F0570
:100080000C945F050C945F050C945F050C945F0560
:100090000C945F050C945F050C945F050C945F0550
:1000A0000C945F050C945F050C945F05720F940F20
:1000B0008210940F8210D90FFC0F8210511064101F
:1000C0004D134D137A137A13D5131114091609160B
:1000D0002914091624152415DF1509160916F51516
:1000E000350C12132B141A8024252680742E2A27EF
:1000F0002122230815171C181E1F202F3031802D98
:1001000039041607090A0B0D0E0F33343228807C90
:1001100079781D1B0619051110363738757D647AFC
:100120002C7B7F8040413A535455565F6061578025
:100130005C5D5E6642433C585A5B67296263598046
:10014000808080803B473D518080494A4B4C4D4EDA
:10015000463E48804452453F504F8080808080809A
:10016000253032583A20253038620A000A722F634F
:100170002030313233343536370A00253032580AD0
:1001800000253032580A004572726F723A202530CD
:1001900032580A00456E640A0073253032583A72AC
:1001A000253032582000456E61626C6520627265B0
:1001B000616B3A20004B6579626F6172642049443B
:1001C0003A20253032580A0049424D203437303425
:1001D00020636F6E7665727465720A00726275666E
:1001E0003A2066756C6C0A00523A25303258253038
:1001F00032580A00533A2530325820005B735D00B4
:100200004B6579626F6172642073746172742E0A37
:100210000055534220636F6E666967757265642E80
:100220000A005B575D005B535D005B525D005B4401
:100230005D005B435D003803490042004D00200033
:10024000340037003000340020006B006500790076
:1002500062006F00610072006400200063006F00A4
:100260006E00760065007200740065007200000088
:100270000E0374002E006D002E006B002E00000097
:100280000403090409027400040100A032090400F7
:1002900000010301010009211101000122400007B2
:1002A00005810308000A0904010001030102000995
:1002B0002111010001224D000705820308000A09EF
:1002C000040200010300000009211101000122368F
:1002D000000705830308000A090403000203000065
:1002E00000092111010001222200070584032000DA
:1002F000010705040320000112011001000000089D
:10030000EDFE07470100010200010631FF0974A15B
:10031000010975150026FF009520750881020976F0
:10032000150026FF00952075089102C0050109807F
:10033000A101850216810026B7001A81002AB700A4
:10034000751095018100C0050C0901A101850316F6
:100350000100269C021A01002A9C02751095018159
:1003600000C005010902A1010901A1000509190147
:100370002905150025019505750181029501750373
:1003800081010501093009311581257F9502750824
:10039000810609381581257F950175088106050CB0
:1003A0000A38021581257F950175088106C0C005B0
:1003B000010906A101050719E029E71500250195A6
:1003C0000875018102950175088101050819012947
:1003D00005950575019102950175039101050719B0
:1003E0000029FF150026FF00950675088100C00A48
:1003F000002530325820006B6579626F6172645F4E
:100400007265706F72743A20004C45443A20253072
:1004100032580A00290A002575002F002575005D55
:1004200028002564002000256400200025640020A9
:10043000002564007C0025303258006D6F757365AF
:100440006B6579205B62746E7C78207920762068F9
:100450005D287265702F61636C293A205B006D6BBB
:100460005F776865656C5F74696D655F746F5F6DFC
:100470006178203D2025640A006D6B5F77686565B3
:100480006C5F6D61785F7370656564203D202564E5
:100490000A006D6B5F74696D655F746F5F6D617885
:1004A000203D2025640A006D6B5F6D61785F73707D
:1004B000656564203D2025640A006D6B5F696E747C
:1004C000657276616C203D2025640A006D6B5F6467
:1004D000656C6179203D2025640A006D6B5F77684B
:1004E00065656C5F74696D655F746F5F6D617820C1
:1004F0003D2025640A006D6B5F776865656C5F6DF4
:1005000061785F7370656564203D2025640A006D25
:100510006B5F74696D655F746F5F6D6178203D20FE
:1005200025640A006D6B5F6D61785F73706565644B
:10053000203D2025640A006D6B5F696E74657276DC
:10054000616C203D2025640A006D6B5F64656C6101
:1005500079203D2025640A000A00257500363A20DE
:10056000776865656C5F74696D655F746F5F6D61F9
:10057000783A20000A00257500353A2077686565CD
:100580006C5F6D61785F73706565643A20000A0086
:10059000257500343A2074696D655F746F5F6D6115
:1005A000783A20000A00257500333A206D61785FA3
:1005B00073706565643A20000A00257500323A20A0
:1005C000696E74657276616C286D73293A20000A31
:1005D00000257500313A2064656C6179282A313034
:1005E0006D73293A20000A092D2056616C756573D8
:1005F000202D0A004D3E004D25643E20003F007333
:1006000065742064656661756C740A00433E200061
:1006100077686572652064656C74613A20637572F1
:10062000736F723D25642C20776865656C3D256489
:100630000A53656520687474703A2F2F656E2E77A3
:10064000696B6970656469612E6F72672F77696B7A
:10065000692F4D6F7573655F6B6579730A000A09C1
:100660002D204D6F7573656B6579202D0A455343B9
:100670002F713A09717569740A313A0964656C61C0
:1006800079282A31306D73290A323A09696E746506
:100690007276616C286D73290A333A096D61785F4F
:1006A00073706565640A343A0974696D655F746FC7
:1006B0005F6D61780A353A09776865656C5F6D61D1
:1006C000785F73706565640A363A09776865656CAA
:1006D0005F74696D655F746F5F6D61780A0A703A67
:1006E000097072696E742076616C7565730A643A7C
:1006F000097365742064656661756C74730A75703E
:100700003A092B310A646F776E3A092D310A706706
:1007100075703A092B31300A7067646F776E3A0949
:100720002D31300A0A7370656564203D2064656C64
:100730007461202A206D61785F7370656564202A7A
:100740002028726570656174202F2074696D655F63
:10075000746F5F6D6178290A003F004D3E200043B1
:100760003E20004C25640A000A092D20436F6E7359
:100770006F6C65202D0A4553432F713A09717569D5
:10078000740A6D3A096D6F7573656B65790A000AB5
:10079000092D204D61676963202D0A643A0964655B
:1007A0006275670A783A096465627567206D6174DD
:1007B0007269780A6B3A096465627567206B6579BE
:1007C000626F6172640A6D3A096465627567206DD3
:1007D0006F7573650A763A0976657273696F6E0A8A
:1007E000733A097374617475730A633A09636F6EBF
:1007F000736F6C65206D6F64650A302D343A096C37
:1008000061796572302D34284631302D4634290AFD
:10081000506175733A09626F6F746C6F61646572D1
:100820000A003F0074696D65725F726561643332FE
:1008300028293A202530346C580A006B6579626F9C
:100840006172645F69646C653A2025580A006B65C3
:1008500079626F6172645F70726F746F636F6C3A0C
:100860002025580A00686F73745F6B6579626F6149
:1008700072645F6C65647328293A2025580A000A5F
:10088000092D20537461747573202D0A004743436A
:100890003A20342E392E32204156522D4C494243B3
:1008A0003A20312E382E3073766E204156525F41F9
:1008B0005243483A20617672350A004F5054494FEE
:1008C0004E533A204C554641204D4F5553454B45CC
:1008D000592045585452414B455920434F4E534F90
:1008E0004C4520434F4D4D414E44204B45594D41C1
:1008F000505F53454354494F4E20343039360A0037
:100900004255494C443A20383030653963612D6492
:1009100069727479202831303A35313A30322053B7
:1009200065702033302032303136290A0056494470
:100930003A2030784645454428742E6D2E6B2E297A
:10094000205049443A203078343730372849424DD6
:100950002034373034206B6579626F6172642063B4
:100960006F6E76657274657229205645523A203052
:1009700078303030310A00444553433A20636F6E7B
:10098000766572742049424D2034373034206B65CF
:1009900079626F61726420746F205553420A000AB5
:1009A000092D2056657273696F6E202D0A000A6D3D
:1009B0006F7573653A206F66660A000A6D6F75730E
:1009C000653A206F6E0A000A6B6579626F61726426
:1009D0003A206F66660A000A6B6579626F6172641D
:1009E0003A206F6E0A000A6D61747269783A206F5E
:1009F00066660A000A6D61747269783A206F6E0A41
:100A0000000A64656275673A206F6E0A000A6465C1
:100A10006275673A206F66660A000A0A626F6F7431
:100A20006C6F616465722E2E2E2000433E20000004
:100A300011241FBECFEFDAE0DEBFCDBF04B603FE48
:100A400027C08091F7019091F801A091F901B09130
:100A5000FA018730904BA740B04BD1F41092F701C8
:100A60001092F8011092F9011092FA0114BE84B7A5
:100A7000877F84BF0FB6F894A89580916000886145
:100A800080936000109260000FBEE0E0F8E30995EB
:100A900011E0A0E0B1E0E2E8FAE402C005900D92B6
:100AA000A233B107D9F721E0A2E3B1E001C01D9262
:100AB000A73FB207E1F70E94620B0C943F250C940C
:100AC0000000FF93EF93E0913201F09133013097F2
:100AD00009F00995EF91FF910895FC01859180300F
:100AE00011F0EFDFFBCF0895FF27E0E230E247FF90
:100AF0000CC0419597FF09C0EDE260957095809517
:100B00009095611D711D811D911D27FF02C02195CA
:100B100030E350E2AA27660F771F881F991FAA1F8C
:100B2000A41710F0A41B63955A95A9F7AA3008F0F2
:100B3000A95FA05DAF93F3956115710581059105DE
:100B400041F7ED3211F4EF93F395F21718F43F9358
:100B5000F395FBCF8F91B5DFFA95E1F70895E99111
:100B6000F9918591803021F0853219F0AADFF9CF13
:100B7000089520E0E89455915532C1F3503311F4B3
:100B8000689455915A3348F4505390F3220F022E33
:100B9000220F220F200D250FF4CF0EF421958991FD
:100BA0009991533619F3533729F1533559F1BC0153
:100BB00088279927E8945C3621F489919991689463
:100BC0005591543639F446EF7EF077FF0DC08FEF24
:100BD0009FEF0AC055374AE039F0583540E121F01F
:100BE000523642E009F00895FF93EF937DDFEF91D5
:100BF000FF91B7CFFF93EF93FC0181918030B9F360
:100C000060DFFBCFFF93EF9368DFF1CFDF93CF93EC
:100C1000CDB7DEB72596A3DFCF91DF9108950C9471
:100C20007307FF920F931F93CF93DF938091D901A6
:100C300081608093D90188EC91E00E946D05E4E326
:100C4000F1E080E18E0F11928E13FDCF2FEF87EA36
:100C500091E6215080409040E1F700C000000E94E2
:100C600048081F928F9385EB91E09F938F930E948A
:100C7000060686EA91E00E946D050F900F900F9096
:100C80000F908CEF0E948207882339F08FE39CE954
:100C90000197F1F700C00000F4CFC0E0D0E009E90F
:100CA00011E08C2F8068F82E8F2D0E9482078823F8
:100CB00039F08FE39CE90197F1F700C00000F4CF11
:100CC0008FE19EE40197F1F700C000000E94480800
:100CD0001F928F93DF93CF931F930F930E9406066B
:100CE00021960F900F900F900F900F900F90CF378D
:100CF000D105B9F68FEF0E948207882339F08FE380
:100D00009CE90197F1F700C00000F4CF84E991E07D
:100D1000DF91CF911F910F91FF900C946D05CF93B0
:100D2000DF930E9448088F3F11F480E05BC0982F4A
:100D30009F779C37A0F01F928F9387E891E09F9355
:100D40008F930E9406060F900F900F900F90E4E390
:100D5000F1E080E18E0F11928E13FDCFE6CF9091DE
:100D6000D901C82FC695C695C695D82FD77087FFCD
:100D70001CC090FF0CC01F928F9381E891E09F935D
:100D80008F930E9406060F900F900F900F90EC2FFC
:100D9000EF70F0E0EC5CFE4F81E090E001C0880F66
:100DA000DA95EAF79081892B1BC090FF0CC01F9247
:100DB0008F938BE791E09F938F930E9406060F908D
:100DC0000F900F900F90EC2FF0E0EC5CFE4F81E065
:100DD00090E001C0880FDA95EAF780959081892329
:100DE000808381E0DF91CF910895E82FF0E0EC5C03
:100DF000FE4F80810895EF92FF920F931F93CF9340
:100E0000DF938CE691E00E946D0584E3E82E81E09B
:100E1000F82EC0E0D0E000E611E0F70181917F01FB
:100E20000E94F31B1F928F93DF93CF931F930F9317
:100E30000E94060621960F900F900F900F900F9032
:100E40000F90C031D10549F7DF91CF911F910F91DC
:100E5000FF90EF90089508959FB7F894209148016E
:100E600080914901821761F030E0F901E65BFE4FA5
:100E700080812F5F3F4F2F7133272093480101C09E
:100E800080E09FBF08955198599A08955898509AB4
:100E900008955098589A08955198599A85E08A95DE
:100EA000F1F7000089B18695817008955098589A9D
:100EB00085E08A95F1F7000089B181700895CF939C
:100EC000DF93C4E6D0E00E944C07811108C0209750
:100ED00031F085E08A95F1F700002197F4CFCE013B
:100EE000DF91CF9108950E9443070E944607E9E6EB
:100EF000F0E080818C608083E19AE99A0E94430748
:100F00000C944907BF92CF92DF92EF92FF920F931A
:100F10001F93CF93DF93C82E10924701E9980E9448
:100F200043070E9449075998519A0CE211E00E9428
:100F3000560781110AC00115110549F085E08A950F
:100F4000F1F7000001501109F2CF012B11F480E3F9
:100F500073C000E010E0D1E0D12CBB24B394C02FCB
:100F60000E945F07892B11F4C05C24C0C601002ECB
:100F700002C0959587950A94E2F780FF04C0DB25AF
:100F80000E94490702C00E94460784E6E82EF12C21
:100F90000E944C07882359F0E114F10451F085E0D8
:100FA0008A95F1F7000081E0E81AF108F1CFEF2807
:100FB00021F4C85BC09347014AC00F5F1F4F083040
:100FC000110569F60E945F07892B11F484E334C090
:100FD000DD2329F00E94490704E610E00CC00E94BE
:100FE0004607FACF0115110561F085E08A95F1F702
:100FF0000000015011090E944C078111F3CF012B11
:1010000011F485E319C00E945F07892BF9F20E9451
:10101000490704E610E00E945607882351F00115A5
:10102000110549F085E08A95F1F70000015011099A
:10103000F2CF012B21F486E38093470108C00E9480
:1010400043070E944907E19AE99A80E017C00E948D
:1010500043070E94490780914701813360F01F9246
:101060008F9384EF91E09F938F930E9406060F90D9
:101070000F900F900F90E19AE99A8FEFDF91CF9147
:101080001F910F91FF90EF90DF90CF90BF90089548
:101090002FB7F89490914901809148012FBF981380
:1010A0000C942C078FEF08951F920F920FB60F929A
:1010B00011242F933F934F935F936F937F938F935D
:1010C0009F93AF93BF93CF93DF93EF93FF931092D0
:1010D0004701809146018830F1F030F0893009F005
:1010E0005CC0C4E6D0E02EC0809145018695809317
:1010F00045010E945607882309F449C080914501A3
:1011000080688093450181E090914401911180E0D5
:10111000809344013CC00E945607882339F081E047
:1011200090914401911180E08093440180914401A9
:10113000882399F12CC0209781F185E08A95F1F7F9
:10114000000021970E9456078111F5CFCD2B29F180
:1011500040914501CFB7F8948091490190E09C01FE
:101160002F5F3F4F2F71332750914801521739F0AD
:10117000FC01E65BFE4F40832093490104C08CEDE7
:1011800091E00E946D05CFBF109247012AC0809167
:1011900046018F5F809346012AC08091460180936B
:1011A00047018EEF0E948207882339F08FE99FE084
:1011B0000197F1F700C00000F4CF809145011F9224
:1011C0008F93809146011F928F9388EE91E09F93B9
:1011D0008F930E9406060F900F900F900F900F9024
:1011E0000F90109246011092450110924401FF9118
:1011F000EF91DF91CF91BF91AF919F918F917F91AF
:101200006F915F914F913F912F910F900FBE0F9073
:101210001F9018958091750108959FB7F8941092CA
:101220006C019FBF9091EE01943009F057C09091EE
:10123000E9009F703091EC00232F217030FD20E8F1
:10124000922B24E02093E9002091EB0020FF43C083
:101250002091EE0027FF3FC020916A01222321F058
:101260002091E80025FF37C010926A0126E03091F6
:10127000E80035FD15C03091EE01343061F5309154
:10128000EB0035FD28C0215021F481E080936A01F4
:1012900022C0EFE9FFE03197F1F700C00000E7CF8F
:1012A0008093F1008091E80085FD0AC08091E800FC
:1012B00080FFFCCF8091E8008E778093E80006C025
:1012C0008FB7F89421E020936C018FBF9F709093AB
:1012D000E90080E008959F709093E9008FEF0895F2
:1012E000CF93DF9300D01F92CDB7DEB79C018091E2
:1012F000EE01843019F593E099833B832A83909320
:10130000E9008FEF9091E800815095FD06C095EDC2
:101310009A95F1F700008111F5CF8091E80085FFE3
:101320000DC040E050E063E070E0CE0101960E9405
:10133000230C8091E8008E778093E8000F900F9047
:101340000F90DF91CF910895CF93DF9300D01F923C
:10135000CDB7DEB72091EE01243021F522E02983BC
:101360009B838A8383E08093E9008FEF9091E8006C
:10137000815095FD06C095ED9A95F1F70000811119
:10138000F5CF8091E80085FF0DC040E050E063E0BC
:1013900070E0CE0101960E94230C8091E8008E77C8
:1013A0008093E8000F900F900F90DF91CF910895F8
:1013B0002091EE012430F1F422E02093E9002FEF98
:1013C0003091E800215035FD06C035ED3A95F1F732
:1013D00000002111F5CF2091E80025FF0BC040E06F
:1013E00050E065E070E00E94230C8091E8008E7769
:1013F0008093E8000895CF93DF932091EE0124308D
:1014000039F521E02093E9002FEF3091E8002150D9
:1014100035FD06C035ED3A95F1F700002111F5CF05
:101420002091E80025FF14C0EC0140E050E068E0A6
:1014300070E00E94230C8091E8008E778093E80092
:1014400088E0FE01ADE6B1E001900D928A95E1F7EA
:10145000DF91CF91089582E392E00E946D05809123
:10146000ED01811109C00E94B80D0E94150E8091F6
:10147000E20084608093E20008958EE292E00E9490
:101480006D051092ED0108958AE292E00C946D05CD
:1014900020916B012F5F822F62E30E940525992323
:1014A00019F020936B01089510926B0180916C01EB
:1014B000882371F18091EE01843041F58091E9003B
:1014C0008F702091EC00922F917020FD90E8892B75
:1014D00094E09093E9009091EB0090FF14C09091FC
:1014E000EE0097FF10C09091E80095FF03C01092A6
:1014F000F100F9CF9091E80090FF05C09091E800CD
:101500009E779093E8008F708093E90010926C01B1
:10151000089542E061EC81E00E94320D42E061EC0E
:1015200082E00E94320D42E061EC83E00E94320DC5
:1015300042E261EC84E00C94320D8091F001833042
:1015400009F453C030F4813071F0823009F48CC05A
:1015500008958A3009F478C08B3009F45EC0893070
:1015600009F09AC020C08091EF01813A09F094C03F
:101570008091E800877F8093E8008091F30190914B
:10158000F401892B21F468E08DE691E003C060E06E
:1015900080E090E070E00E946E0C8091E8008B7714
:1015A0008093E80008958091EF01813209F074C0C2
:1015B0008091F3019091F401892B09F06DC0809125
:1015C000E800877F8093E8008091E80082FD05C0F5
:1015D0008091EE018111F8CF5FC08091F10080937E
:1015E00075018091E8008B7753C08091EF01813ABB
:1015F00009F052C08091F3019091F401892B09F018
:101600004BC08091E800877F8093E8008091E800DC
:1016100080FFFCCF80910A0136C08091EF018132BA
:10162000D9F58091F3019091F401892BA9F580916E
:10163000E800877F8093E8000E94670D8091F101A8
:1016400080930A010C942A168091EF01813221F5D2
:101650008091E800877F8093E8000E94670D809169
:10166000F2018093760108958091EF01813AA1F40F
:101670008091E800877F8093E8008091E80080FFF8
:10168000FCCF809176018093F1008091E8008E7705
:101690008093E8000C94670D0895089508950895C7
:1016A00086E292E00E946D050C944F0B0E941D1C77
:1016B0008091EC01882329F00E94481C81110C9430
:1016C0000D0C089584B7877F84BF0FB6F894A89552
:1016D00080916000886180936000109260000FBE6E
:1016E00090E080E80FB6F8948093610090936100D9
:1016F0000FBE0E944D0B0E942B110E94B80D0E943C
:10170000150E8091E20084608093E2008DE099E004
:101710000E94EE1B78948091EE018430E1F781E124
:1017200092E00E946D050E942D1180E091E00E94E0
:101730009A1080E092E00E946D050E944E0B80910D
:10174000EE01853039F48CEF91E00E946D050E9426
:10175000560BF5CF0E943111F2CF0C945C1C82E243
:1017600092E00E946D050C94AD0B292F3327233096
:101770003105C9F064F42130310581F022303105A2
:1017800009F043C084E790E024E832E042C021320F
:101790003105F1F02232310541F137C082E190E0AC
:1017A00028EF32E036C099278130910541F0823030
:1017B000910541F0892B49F5E0E8F2E005C0E0E74A
:1017C000F2E002C0E6E3F2E0849190E09F0121C0E4
:1017D0006430D8F4E62FF0E0EE0FFF1FE15EFE4F1D
:1017E0002081318189E090E014C0643070F470E0B1
:1017F000FB01EE0FFF1FE95EFE4F20813181FB01EF
:10180000ED5EFE4F808190E004C080E090E020E03B
:1018100030E0FA0131832083089580E189BD82E1BF
:1018200089BD09B400FEFDCF8091D8008F7D8093E3
:10183000D8008091E00082608093E0008091E00019
:1018400081FDFCCF0895CF92DF92EF92FF920F932C
:101850001F93CF93DF93EC018B016A010E94860DE9
:10186000811133C0C114D10439F0F6018081918116
:10187000081B190BC80FD91FE12CF12C01151105FC
:1018800019F18091E80085FD16C08091E8008E77FF
:101890008093E800C114D10449F0F6018081918160
:1018A000E80EF91EF182E08285E00FC00E94860DED
:1018B000882321F30AC089918093F1000150110916
:1018C000FFEFEF1AFF0ADACF80E0DF91CF911F918F
:1018D0000F91FF90EF90DF90CF9008952091F50148
:1018E0003091F6012617370748F06115710539F474
:1018F0002091E8002E772093E80001C0B90140E074
:1019000061157105A9F12091EE01222309F443C06C
:10191000253009F442C02091E80023FD40C0209109
:10192000E80022FD32C02091E80020FFE9CF40917D
:10193000F3002091F20030E0342BFC01CF0161155F
:10194000710559F02830310540F481918093F10000
:10195000615071092F5F3F4FF1CF41E028303105D1
:1019600009F040E02091E8002E772093E800C8CFEE
:101970004111C9CF0AC08091EE01882361F0853002
:1019800061F08091E80083FD0AC08091E80082FF49
:10199000F2CF80E0089582E0089583E0089581E029
:1019A00008952091F5013091F6012617370748F088
:1019B0006115710539F42091E8002E772093E80035
:1019C00001C0B901FC0120E06115710591F1809120
:1019D000EE01882309F440C0853009F43FC08091AE
:1019E000E80083FD3DC08091E80082FD2FC080911A
:1019F000E80080FFE9CF2091F3008091F20090E0B1
:101A0000922B6115710559F08830910540F42491AD
:101A10002093F1003196615071090196F2CF21E0D7
:101A2000089709F020E08091E8008E778093E80025
:101A3000CBCF2111CCCF0AC08091EE01882361F079
:101A4000853061F08091E80083FD0AC08091E80054
:101A500082FFF2CF80E0089582E0089583E0089548
:101A600081E00895982F973058F59093E9009817E2
:101A700039F07091EC002091ED005091F00003C01E
:101A8000242F762F50E021FF19C03091EB003E7FCC
:101A90003093EB003091ED003D7F3093ED003091BD
:101AA000EB0031603093EB007093EC002093ED007D
:101AB0005093F0002091EE0027FF07C09F5FD3CF27
:101AC0008F708093E90081E0089580E0089580910F
:101AD000EF0187FF11C08091E80082FD05C0809171
:101AE000EE018111F8CF11C08091E8008B770BC017
:101AF0008091EE01882349F08091E80080FFF8CFC3
:101B00008091E8008E778093E80008952091E400AA
:101B10003091E50095E64091EC00842F817040FF04
:101B200022C08091E80080FD1CC08091EE018823D6
:101B300091F0853091F08091EB0085FD10C04091CF
:101B4000E4005091E5004217530729F39A019150A0
:101B500011F784E0089582E0089583E0089581E01C
:101B6000089580E008954091E80042FFDECF089597
:101B70000E94260E0E942E0EE0EEF0E08081816031
:101B80008083E8EDF0E080818F77808319BCA7ED3A
:101B9000B0E08C918E7F8C9380818F7E80831092B9
:101BA000ED0108950F931F93CF93DF930E94260EAC
:101BB0000E942E0EC8EDD0E088818F7788838881BF
:101BC0008068888388818F7D888319BC1092EE019C
:101BD0001092EA011092EC011092EB0100EE10E07D
:101BE000F80180818B7F808388818160888342E0D7
:101BF00060E080E00E94320DE1EEF0E080818E7FB7
:101C00008083E2EEF0E08081816080838081886063
:101C10008083F80180818E7F8083888180618883C2
:101C2000DF91CF911F910F910895E8EDF0E0808151
:101C30008F7E8083E7EDF0E080818160808384E0A7
:101C400082BF81E08093ED010C94D20DE8EDF0E0CD
:101C500080818E7F80831092E20008951092DA00D6
:101C60001092E10008951F920F920FB60F92112467
:101C70002F933F934F935F936F937F938F939F9394
:101C8000AF93BF93EF93FF938091E10082FF0BC06E
:101C90008091E20082FF07C08091E1008B7F8093FA
:101CA000E1000E94480A8091DA0080FF1FC0809105
:101CB000D80080FF1BC08091DA008E7F8093DA000D
:101CC0008091D90080FF0DC080E189BD82E189BD8E
:101CD00009B400FEFDCF81E08093EE010E942B0A43
:101CE00005C019BC1092EE010E943D0A8091E100EE
:101CF00080FF19C08091E20080FF15C08091E20052
:101D00008E7F8093E2008091E20080618093E20008
:101D10008091D80080628093D80019BC85E08093C0
:101D2000EE010E94500B8091E10084FF30C0809151
:101D3000E20084FF2CC080E189BD82E189BD09B445
:101D400000FEFDCF8091D8008F7D8093D8008091D8
:101D5000E1008F7E8093E1008091E2008F7E80938E
:101D6000E2008091E20081608093E2008091EA01CC
:101D7000882311F084E007C08091E30087FD02C052
:101D800081E001C083E08093EE010E94AF0B80915F
:101D9000E10083FF29C08091E20083FF25C080918C
:101DA000E100877F8093E10082E08093EE01109252
:101DB000EA018091E1008E7F8093E1008091E20052
:101DC0008E7F8093E2008091E20080618093E20048
:101DD00042E060E080E00E94320D8091F000886077
:101DE0008093F0000E94440AFF91EF91BF91AF9160
:101DF0009F918F917F916F915F914F913F912F9123
:101E00000F900FBE0F901F9018951F920F920FB654
:101E10000F9211242F933F934F935F936F937F9370
:101E20008F939F93AF93BF93CF93DF93EF93FF93E2
:101E3000C091E900CF708091EC00D82FD17080FD67
:101E4000D0E81092E9008091F000877F8093F00045
:101E500078940E94490F1092E9008091F000886008
:101E60008093F000CD2BCF70C093E900FF91EF91EC
:101E7000DF91CF91BF91AF919F918F917F916F91A2
:101E80005F914F913F912F910F900FBE0F901F9038
:101E900018951F93CF93DF93CDB7DEB7AA970FB6F0
:101EA000F894DEBF0FBECDBFEFEEF1E088E08E0FFD
:101EB0009091F10091938E13FBCF0E949D0A809127
:101EC000E80083FF1FC18091EF019091F001492F3D
:101ED00050E04A30510508F015C1FA01EA5AFF4FA7
:101EE0000C942525803881F0823809F00BC180914F
:101EF000F3018F708093E9008091EB0085FB8827C8
:101F000080F91092E90006C08091EB019091EC01FC
:101F1000911182609091E800977F9093E800809300
:101F2000F1001092F100C8C0282F2D7F09F0EAC0FF
:101F3000882319F0823061F0E5C08091F101813091
:101F400009F0E0C0933009F080E08093EC012BC0F1
:101F50008091F101811127C08091F3018F7009F404
:101F6000D1C08093E9002091EB0020FF1CC093308A
:101F700021F48091EB00806214C09091EB0090619D
:101F80009093EB0021E030E0A90102C0440F551FFF
:101F90008A95E2F74093EA001092EA008091EB0004
:101FA00088608093EB001092E9008091E800877FC1
:101FB00086C08111A7C01091F1011F778091E300C5
:101FC0008078812B8093E3008091E800877F809365
:101FD000E8000E94670D8091E80080FFFCCF8091AF
:101FE000E30080688093E300111102C082E001C029
:101FF00083E08093EE0186C08058823008F082C072
:102000008091F1019091F2018C3D53E0950779F5B3
:1020100083E08A838AE289834FB7F894DE011396BE
:1020200020E03EE051E2E32FF0E050935700E491CE
:1020300020FF03C0E295EF703F5FEF708E2F90E0BE
:10204000EA3010F0C79601C0C0968D939D932F5F24
:10205000243149F74FBF8091E800877F8093E800E3
:102060006AE270E0CE0101960E946E0C14C0AE01CF
:102070004F5F5F4F6091F3010E94B50BBC01892B4C
:1020800009F440C09091E800977F9093E80089811F
:102090009A810E94D10C8091E8008B778093E800B0
:1020A00031C0803879F58091E800877F8093E8001F
:1020B0008091EA018093F1008091E8008E7780930F
:1020C000E8000E94670D1EC081111CC09091F101B3
:1020D0009230C0F48091E800877F8093E80090936D
:1020E000EA010E94670D8091EA01811106C080918A
:1020F000E30087FD02C081E001C084E08093EE012F
:102100000E94890A8091E80083FF0AC08091E8005C
:10211000877F8093E8008091EB0080628093EB00E2
:10212000AA960FB6F894DEBF0FBECDBFDF91CF9158
:102130001F91089590937C0180937B010895E09115
:102140007B01F0917C01309721F00190F081E02D2E
:10215000099480E00895EF92FF920F931F93CF931D
:10216000DF93E0917B01F0917C013097B1F18C011C
:102170000280F381E02D09958091D90182FF2DC065
:1021800080FF04C087EF93E00E946D05E80118E02E
:1021900081EFE82E83E0F82E8091D90180FF0BC0FB
:1021A00088811F928F93FF92EF920E9406060F90F4
:1021B0000F900F900F90115021961111EDCF80913B
:1021C000D90180FF0AC08FEE93E0DF91CF911F917C
:1021D0000F91FF90EF900C946D05DF91CF911F91BF
:1021E0000F91FF90EF900895E0917B01F0917C01B9
:1021F000309721F00480F581E02D09940895209115
:10220000790130917A018217930771F090937A01E6
:1022100080937901E0917B01F0917C01309721F06E
:102220000680F781E02D099408952091770130917F
:1022300078018217930771F090937801809377016A
:10224000E0917B01F0917C01309721F00084F185D1
:10225000E02D099408950C940F060E94871C0C949D
:102260001106CF92DF92EF92FF920F931F93CF93BD
:10227000DF9300D000D000D0CDB7DEB70E948F062C
:102280008EE7C82E81E0D82E00E010E0E02E802FEF
:102290000E94F506F60141916F01F42EF826B1F483
:1022A0000F5F1F4F0031110589F78FEF89838A83F4
:1022B0001B820E94901C8160782F9D838C834981B2
:1022C0005A816B818D810E94F01147C09091D90194
:1022D00091FF04C08E830E94FB068E8120E030E0D7
:1022E0004F2D50E0922FBA01022E02C075956795CE
:1022F0000A94E2F760FF2BC02983EA8221E030E0F4
:10230000690102C0CC0CDD1C9A95E2F790E08C21AB
:102310009D21892B09F420E02B830E94901C816071
:10232000782F9D838C8349815A816B818D810E9496
:10233000F01149815A816B817C818D810E940A1C38
:10234000F801E258FE4F8081C826C08206C02F5F88
:102350003F4F2830310531F6A3CF0E94091C0E945F
:10236000511F10917D010E949F10181741F10E948A
:102370009F1080937D019091D90192FF0EC090FF34
:102380000CC01F928F9389E094E09F938F930E94DB
:1023900006060F900F900F900F9080917D0126966A
:1023A0000FB6F894DEBF0FBECDBFDF91CF911F9166
:1023B0000F91FF90EF90DF90CF900C941B1C26960E
:1023C0000FB6F894DEBF0FBECDBFDF91CF911F9146
:1023D0000F91FF90EF90DF90CF9008950C942B0712
:1023E000CF93DF93CDB7DEB72B970FB6F894DEBF50
:1023F0000FBECDBF942F4F83252F588769877A87CB
:102400008B874A855B85452B21F02F3F09F59F3F40
:10241000F9F4DE01119686E0FD0111928A95E9F743
:1024200085E0FE01379601900D928A95E1F749818A
:102430005A816B817C818D819E810E94C4182B966C
:102440000FB6F894DEBF0FBECDBFDF91CF910895D8
:102450004F81588569857A858B850E940A1CD9CF62
:10246000CF93882309F4A4C0C82F8CEF8C0F813A36
:1024700048F48C2F0E947B2281119AC08C2F0E94DD
:102480004F1B0CC080E28C0F883058F4C77081E07D
:1024900001C0880FCA95EAF70E948E1BCF910C9459
:1024A000C81B8BE58C0F833078F4C53A29F0C63A07
:1024B00031F083E890E005C081E890E002C082E856
:1024C00090E0CF910C94FF1088E58C0F853108F0D7
:1024D0006FC0C83A61F1C93A69F1CA3A71F1CB3AB1
:1024E00079F1CC3A81F1CD3A89F1CE3A91F1CF3AF6
:1024F00099F1C13BA1F1C03BA9F1C23BB1F1C33B92
:10250000B9F1C43BC1F1C53BC9F1C63BD1F1C73BF1
:10251000D9F1C83BE1F1C93BE9F1CA3BF1F1CB3B51
:10252000F9F1CC3B09F43FC080E090E03EC082EE80
:1025300090E03BC089EE90E038C08AEE90E035C074
:1025400085EB90E032C086EB90E02FC083EB90E00B
:102550002CC084EB90E029C087EB90E026C08CEC87
:1025600090E023C08DEC90E020C083E891E01DC096
:102570008AE891E01AC082E991E017C084E991E00D
:1025800014C081E292E011C083E292E00EC084E2C6
:1025900092E00BC085E292E008C086E292E005C0BE
:1025A00087E292E002C08AE292E0CF910C9415118A
:1025B000CF910895882329F19CEF980F913A18F450
:1025C0000E946C1B0DC090E2980F983058F48770F1
:1025D00091E001C0990F8A95EAF7892F0E94941B18
:1025E0000C94C81B9BE5980F933020F480E090E09A
:1025F0000C94FF10885A853120F480E090E00C9410
:1026000015110895882321F00E948E1B0C94C81B7D
:102610000895882321F00E94941B0C94C81B0895F0
:10262000CF92DF92EF92FF920F931F93CF93DF939E
:1026300000D000D000D0CDB7DEB725E0FC01DE0130
:10264000119601900D922A95E1F7FC0140813181AC
:10265000F280258122952F7063817481672B09F4A4
:10266000D8C23F3F19F44F3F09F4D3C26C014983EC
:102670003A8389819A812E830E940E1B182F092F7D
:102680000E940D1B0E941D1AE02FE295EF70F0E0F2
:10269000E05AFF4F2E810C942525802F807F902FAC
:1026A0009F70092F882311F00295007FFF2049F0C9
:1026B000002309F45FC2802F0E94A11B0E94C81B47
:1026C00059C2812F0E94DA12002309F4A2C2802F7E
:1026D0000E94A71B26960FB6F894DEBF0FBECDBF93
:1026E000DF91CF911F910F91FF90EF90DF90CF90EE
:1026F0000C94C81B802F807F902F9F70092F8032F1
:1027000011F00295007F112319F0113001F129C059
:10271000FF20A9F0802F222349F1213039F5269698
:102720000FB6F894DEBF0FBECDBFDF91CF911F91E2
:102730000F91FF90EF90DF90CF900C94B11B22236C
:1027400019F0213009F465C20E94B41B2CC0FF208F
:10275000E9F0263008F05DC20E948B1B802329F02F
:1027600022C0FF20F1F0211115C0802F26960FB650
:10277000F894DEBF0FBECDBFDF91CF911F910F91B7
:10278000FF90EF90DF90CF900C940213253008F06B
:1027900040C209C0F601858180FFECC18F7085833E
:1027A000E4CF2111FBC1802F69C1202F26952695EA
:1027B000237030E02115310521F021303105C9F0B9
:1027C00028C2FF2021F0812F902F937002C080E05B
:1027D00090E026960FB6F894DEBF0FBECDBFDF9116
:1027E000CF911F910F91FF90EF90DF90CF900C94BD
:1027F000FF10FF2021F0812F902F937002C080E006
:1028000090E026960FB6F894DEBF0FBECDBFDF91E5
:10281000CF911F910F91FF90EF90DF90CF900C948C
:102820001511812FFF2019F00E94D71D02C00E94B0
:102830003F1E26960FB6F894DEBF0FBECDBFDF91C8
:10284000CF911F910F91FF90EF90DF90CF900C945C
:10285000C41E802F837009F078C0F110DAC1812F77
:10286000829586958770880F880F912F9F70C92E4B
:10287000D12CE12CF12C082E04C0CC0CDD1CEE1C5C
:10288000FF1C0A94D2F714FF12C04FE050E060E042
:1028900070E004C0440F551F661F771F8A95D2F75A
:1028A000CB01BA01609570958095909503C060E06A
:1028B00070E0CB01202F269526952370422F50E003
:1028C00042305105D1F04330510559F16C297D2931
:1028D0008E299F294130510541F126960FB6F89473
:1028E000DEBF0FBECDBFDF91CF911F910F91FF9043
:1028F000EF90DF90CF900C94321A6C297D298E29AD
:102900009F2926960FB6F894DEBF0FBECDBFDF918C
:10291000CF911F910F91FF90EF90DF90CF900C948B
:10292000441A0E94321AC701B60126960FB6F894CF
:10293000DEBF0FBECDBFDF91CF911F910F91FF90F2
:10294000EF90DF90CF900C94201AFF2019F0802F89
:10295000817001C08695882309F45BC1812F82951F
:1029600086958770880F880F912F9F70C92ED12C64
:10297000E12CF12C082E04C0CC0CDD1CEE1CFF1C3D
:102980000A94D2F714FF12C04FE050E060E070E00C
:1029900004C0440F551F661F771F8A95D2F7CB01DD
:1029A000BA01609570958095909503C060E070E0E5
:1029B000CB01202F269526952370422F50E04230E0
:1029C0005105D1F04330510559F16C297D298E29EB
:1029D0009F294130510541F126960FB6F894DEBF8C
:1029E0000FBECDBFDF91CF911F910F91FF90EF9060
:1029F000DF90CF900C94E91A6C297D298E299F29AC
:102A000026960FB6F894DEBF0FBECDBFDF91CF91F3
:102A10001F910F91FF90EF90DF90CF900C94FB1AD5
:102A20000E94E91AC701B60126960FB6F894DEBFD8
:102A30000FBECDBFDF91CF911F910F91FF90EF900F
:102A4000DF90CF900C94D71A103F41F118F4103E4C
:102A500048F48BC0123F09F450C0D8F1133F09F479
:102A600060C083C01F70802F8F71FF2021F00E94F3
:102A7000701A812F7BCE0E94911A812F26960FB655
:102A8000F894DEBF0FBECDBFDF91CF911F910F91A4
:102A9000FF90EF90DF90CF900C940913FF20A9F0E6
:102AA000253008F0B6C0802F8F7126960FB6F894A7
:102AB000DEBF0FBECDBFDF91CF911F910F91FF9071
:102AC000EF90DF90CF900C94B61A263008F0A1C09A
:102AD000EACFFF20A1F0802F8F7126960FB6F894D1
:102AE000DEBF0FBECDBFDF91CF911F910F91FF9041
:102AF000EF90DF90CF900C94701AFF2061F3802F3D
:102B00008F7126960FB6F894DEBF0FBECDBFDF9152
:102B1000CF911F910F91FF90EF90DF90CF900C9489
:102B2000911AFF2091F0802F8F7126960FB6F8949E
:102B3000DEBF0FBECDBFDF91CF911F910F91FF90F0
:102B4000EF90DF90CF900C945B1A26960FB6F89416
:102B5000DEBF0FBECDBFDF91CF911F910F91FF90D0
:102B6000EF90DF90CF900C94561AFF20A1F0222313
:102B700009F4B1CF812F26960FB6F894DEBF0FBEB1
:102B8000CDBFDF91CF911F910F91FF90EF90DF901C
:102B9000CF900C943012222309F4B1CF812F2696C6
:102BA0000FB6F894DEBF0FBECDBFDF91CF911F915E
:102BB0000F91FF90EF90DF90CF900C94DA12402F9E
:102BC0004F70612FC6010E94511D26960FB6F894D2
:102BD000DEBF0FBECDBFDF91CF911F910F91FF9050
:102BE000EF90DF90CF900C946819402F4F70612FB9
:102BF000C60126960FB6F894DEBF0FBECDBFDF919B
:102C0000CF911F910F91FF90EF90DF90CF900C9498
:102C1000541D26960FB6F894DEBF0FBECDBFDF91D0
:102C2000CF911F910F91FF90EF90DF90CF9008957B
:102C30000E94AE1B0E947D1B0E94C81B0E94F61FB3
:102C40000E94C41E80E090E00E94FF1080E090E0AF
:102C50000C9415110E949E1B0C9418160E940E1BBA
:102C6000292F22952F7030E02C3031054CF42A307A
:102C700031056CF4225031092230310588F407C047
:102C80002C30310549F02F30310531F009C0803E3C
:102C900048F0803F29F406C093FB882780F9089507
:102CA00080E0089581E00895CF93DF9300D000D0B5
:102CB0001F92CDB7DEB70F900F900F900F900F902F
:102CC000DF91CF910895CF93DF9300D000D000D053
:102CD000CDB7DEB726960FB6F894DEBF0FBECDBFD8
:102CE000DF91CF9108951F93CF93DF93C0918E0111
:102CF00016E080918F01C81799F0D0E01C9FF00179
:102D00001D9FF00D1124E057FE4F408151816281DB
:102D10007381848195810E9463162196C770E9CFE3
:102D2000DF91CF911F9108954091C0015091C10151
:102D30006091C2017091C3018091C4019091C5015D
:102D40000C9463168091C50182958F7009F054C070
:102D50008091C201882309F44FC080918E01A09117
:102D60008F016091C0017091C1014091C3015091E8
:102D7000C401B6E08A1709F43FC090E0411551053F
:102D8000C1F17F3F11F46F3FA1F1B89FF001B99FEE
:102D9000F00D1124E057FE4F218172132AC02081CB
:102DA000621327C02281211124C02381348124177A
:102DB000350710F421503109241B350B283C31050F
:102DC000C0F42091C5012F7020612093C50126E039
:102DD000289FF001299FF00D1124EB56FE4F8081B2
:102DE0008F708061808380EC91E00E9410130C94BE
:102DF000731601968770BECF0895CF92DF92EF923F
:102E0000FF920F931F93CF93DF93CDB7DEB76297F7
:102E10000FB6F894DEBF0FBECDBF8C0185E0F80180
:102E2000DE011D9601900D928A95E1F7D8014C9133
:102E300011965C91119712966C9112971396CD9002
:102E4000DC9014973091C0017091C1018091C30151
:102E50009091C401009709F46BC17F3F19F43F3F83
:102E600009F466C1E090C201EE2009F4C0C02091CF
:102E7000C501C816D90628F0F601E81BF90BCF01E9
:102E800004C0809590958C0D9D1DFF24F394883C83
:102E9000910578F0F12C207F09F0C6C07C2DD98AED
:102EA000C88A89890E94541680EC91E00E94101310
:102EB000B1C0822F807F09F046C0751314C034134F
:102EC00012C0611110C02F7020612093C5010E94B3
:102ED000941680EC91E00E9410138091C501D801F6
:102EE00015968C932EC0CD2819F15F3F11F44F3FFA
:102EF000F9F0F62E61111CC080918E0120918F0196
:102F000036E0821709F45AC090E0389FF001399FEB
:102F1000F00D1124E057FE4F7181571306C07081E8
:102F2000471303C07281711103C001968770E9CF06
:102F3000F62E662309F418C18091C5018160809343
:102F4000C501F12C11C1751308C0341306C06111FD
:102F500004C08091C501D801C3C04D875E878D85AF
:102F60009E856A8B0E942E166A898823E1F166236A
:102F7000D1F12091C501822F82958F7090E0029748
:102F800074F08091C0019091C10198878F83198658
:102F9000DB86CA862C87CE0107960E94101386E036
:102FA000F801A0ECB1E001900D928A95E1F70E9442
:102FB000A2160E949416FF24F394D6C04D875E8714
:102FC0008D859E850E940E1B292F22952F7030E043
:102FD000223031050CF0BCC09F7009F0B6C0805E95
:102FE000883008F4C1C0C8010E941013E4CFC8168D
:102FF000D90608F453C0F601E81BF90BCF01883C51
:10300000910508F450C0F12C7C2DD98AC88A898991
:103010000E945416E0ECF1E086E0DF011D928A95F3
:10302000E9F70E949416A0C0751314C0341312C09F
:10303000611110C08091C501F8018583C8010E940B
:10304000101386E0E0ECF1E0DF011D928A95E9F7CC
:10305000FE2C8AC04D875E878D859E856A8B0E9477
:103060002E166A89882309F4BECF662309F4BBCFE4
:103070002091C501822F82958F7090E002970CF409
:103080008ECF8091C0019091C1019A8389831B8268
:10309000DD82CC822E83CE0101967FCF80959095E4
:1030A0008C0D9D1DACCFF62E662309F49CCF7513B5
:1030B0002EC034132CC02091C50120FD1FC0822FCB
:1030C00082958F70D9F0D80115962C9315978F3073
:1030D00049F08F5F982F9295907F822F8F70892B68
:1030E00015968C93C8010E94101386E0F801A0EC9D
:1030F000B1E001900D928A95E1F793CF86E0F80157
:10310000A0ECB1E001900D928A95E1F72DC04D87BA
:103110005E878D859E850E942E16811140CF8091FD
:10312000C50181608093C501C8010E9410131CC0B5
:10313000662309F458CF4D875E878D859E850E9452
:103140002E16882309F44FCF2ACF811148CF0CC007
:10315000243031050CF047CF9F7009F440CFF801BF
:103160009581907F09F03BCF8F2D62960FB6F89432
:10317000DEBF0FBECDBFDF91CF911F910F91FF90AA
:10318000EF90DF90CF9008951F93CF93DF93CDB74B
:10319000DEB72C970FB6F894DEBF0FBECDBF4F83BE
:1031A000588769877A878B879C87CE0107960E940C
:1031B000FD16882369F08F8198852A853B85232B0E
:1031C000F1F19F3F09F063C08F3F09F060C037C045
:1031D00086E0FE013796DE01119601900D928A95E8
:1031E000E1F76F817885EA85FB85309741F17F3F74
:1031F00011F46F3F21F120918F0130E0C901019658
:103200008770992740918E0150E08417950709F443
:1032100047C069837A83FD83EC8396E0929FD00157
:10322000939FB00D1124A057BE4FFE01319601901F
:103230000D929A95E1F780938F010E94731616E024
:1032400080918E0190918F018917C1F1189FC00163
:10325000112480579E4F0E94FD16882379F1E0913A
:103260008E011E9FF0011124E057FE4F40815181D5
:1032700062817381848195810E94631680918E01A1
:1032800090E001968770992780938E01D9CF4F8166
:10329000588569857A858B859C850E946316CFCF7A
:1032A0000E942A1610928F0110928E01E0ECF1E03C
:1032B00086E0DF011D928A95E9F7C1CF2C960FB603
:1032C000F894DEBF0FBECDBFDF91CF911F9108955F
:1032D000DF92EF92FF920F931F93CF93DF93FC0146
:1032E000892B09F48AC0E12CF12CDD24D394EF0161
:1032F00021968491853709F461C058F4843708F029
:103300004EC0843008F06AC08130D1F0823071F153
:1033100074C0883709F45DC050F4863709F455C08D
:10332000873709F06AC08E2D0E949B1B54C09CE712
:10333000980F903708F061C08F770E94DA1250C062
:103340008F010E5F1F4FFE01849190E2980F98301D
:1033500050F48770FD2D01C0FF0F8A95EAF78F2F7B
:103360000E94A11B14C00E94301213C08F010E5F77
:103370001F4FFE01C49180E28C0F883060F4C7704B
:103380008D2D01C0880FCA95EAF70E94A71B0E94E5
:10339000C81BE80125C08C2F0E94DA12FACF9F01CA
:1033A0002E5F3F4FFE01C491CC2369F08FE99FE06F
:1033B0000197F1F700C00000C150F6CF9F012E5FCA
:1033C0003F4FFE01F490E9010BC00E948B1BE82ED9
:1033D00007C00E949E1B0E94C81B02C00E943012A0
:1033E0008F2D882341F0EFE9FFE03197F1F700C01E
:1033F00000008150F6CFFE017ACFDF91CF911F916F
:103400000F91FF90EF90DF9008956093CA01709341
:10341000CB018093CC019093CD010E94191C0C9498
:1034200018166093C6017093C7018093C8019093EA
:10343000C9010E941A1C0C94181608950C94051AC0
:103440000F931F930091CA011091CB012091CC01E1
:103450003091CD01602B712B822B932B1F910F91FB
:103460000C94051A0F931F930091CA011091CB0180
:103470002091CC013091CD016023712382239323CD
:103480001F910F910C94051A0F931F930091CA017D
:103490001091CB012091CC013091CD016027712793
:1034A000822793271F910F910C94051A60E070E01A
:1034B000CB010C94111A0F931F9341E050E060E090
:1034C00070E08A019B0104C0000F111F221F331FEF
:1034D0008A95D2F7C901B8011F910F910C94111A66
:1034E0000F931F9341E050E060E070E004C0440F90
:1034F000551F661F771F8A95D2F78091C60190915C
:10350000C701A091C801B091C9018A019B01082B94
:10351000192B2A2B3B2BC901B8011F910F910C9439
:10352000111A0F931F9341E050E060E070E004C077
:10353000440F551F661F771F8A95D2F74095509507
:10354000609570958091C6019091C701A091C801C6
:10355000B091C9018A019B01082319232A233B2327
:10356000C901B8011F910F910C94111A0F931F9369
:1035700041E050E060E070E004C0440F551F661F5A
:10358000771F8A95D2F78091C6019091C701A091CB
:10359000C801B091C9018A019B01082719272A2770
:1035A0003B27C901B8011F910F910C94111A0F9379
:1035B0001F930091C6011091C7012091C80130915D
:1035C000C901602B712B822B932B1F910F910C94AF
:1035D000111A0F931F930091C6011091C7012091FA
:1035E000C8013091C90160237123822393231F9165
:1035F0000F910C94111A0F931F930091C601109113
:10360000C7012091C8013091C90160277127822725
:1036100093271F910F910C94111A0895CF92DF9266
:10362000EF92FF920F931F93CF93DF938C01C09083
:10363000CA01D090CB01E090CC01F090CD01409137
:10364000C6015091C7016091C8017091C901C42A97
:10365000D52AE62AF72ACFE1D0E0D701C6010C2E01
:1036600004C0B695A795979587950A94D2F780FFE1
:1036700007C0B8018C2F0E94271D8130910531F4BD
:10368000219758F7B80180E00E94271DDF91CF9164
:103690001F910F91FF90EF90DF90CF9008952091B0
:1036A0000B0130910C01F90132969FEF40E05191EE
:1036B000581789F09F3F19F4511101C0942F4F5FA3
:1036C0004630A9F79F3F39F0F901E90FF11D97FD49
:1036D000FA9582830895089520910B0130910C0191
:1036E000F9013296285F3F4F9081981301C01082F4
:1036F0003196E217F307C1F7089581E090E0E09179
:103700000B01F0910C01E80FF91F1082019688302F
:103710009105A9F708958091D80108959091D80155
:10372000892B8093D801089580959091D8018923A1
:103730008093D80108958093D80108951092D801FC
:1037400008959091D701892B8093D7010895809592
:103750009091D70189238093D70108951092D701C2
:1037600008958093CE0108951092CE01089580911E
:103770000B0190910C01FC0131969C01285F3F4F99
:1037800080E0919191118F5FE217F307D1F70895CF
:10379000E0910B01F0910C018091D8018083E091C0
:1037A0000B01F0910C0190818091D701892B8083CE
:1037B0008091CE01882361F0E0910B01F0910C0122
:1037C0009081892B80830E94B71B81111092CE01BA
:1037D00080910B0190910C010C94AB1090933301EC
:1037E0008093320108958295982F9C7C392F3695CD
:1037F0003695282F237344E0249FC0011124932F72
:10380000982B292F2A7A2695892F8575880F822B48
:1038100008950895CF93DF9300D000D01F92CDB7C5
:10382000DEB70F900F900F900F900F90DF91CF9118
:103830000895089508950C94EE118091EE0184305E
:1038400021F11092DA0120E488E190E00FB6F894BB
:10385000A895809360000FBE2093600083B7817F9E
:10386000846083BF83B7816083BF7894889583B772
:103870008E7F83BF0FB6F894A89580916000886111
:1038800080936000109260000FBE0895089508951F
:10389000CF930E94461C0E948F060E94471CC0E0E6
:1038A0008C2F0E94F506811104C0CF5FC031C1F793
:1038B00001C081E0CF9108950C942A161F920F92B7
:1038C0000FB60F9211248F939F93AF93BF93809164
:1038D000DA01811113C08091DB019091DC01A0918C
:1038E000DD01B091DE014196A11DB11D8093DB0188
:1038F0009093DC01A093DD01B093DE01BF91AF9105
:103900009F918F910F900FBE0F901F90189582E09E
:1039100084BD93E095BD9AEF97BD80936E000895A6
:103920002FB7F8948091DB019091DC01A091DD012B
:10393000B091DE012FBF08952FB7F8946091DB019D
:103940007091DC018091DD019091DE012FBF08951F
:10395000CF92DF92EF92FF920F931F932FB7F894BD
:103960004091DB015091DC016091DD017091DE013D
:103970002FBF6A017B01EE24FF248C0120E030E0A0
:10398000C016D106E206F30610F4415051099A011F
:10399000281B390BC9011F910F91FF90EF90DF9009
:1039A000CF9008951F920F920FB60F9211248F930C
:1039B0009F93AF93BF938091DB019091DC01A09125
:1039C000DD01B091DE010196A11DB11D8093DB01E7
:1039D0009093DC01A093DD01B093DE01BF91AF9124
:1039E0009F918F910F900FBE0F901F9018950E947E
:1039F000B80DF8942FEF87EA91E62150804090406F
:103A0000E1F700C0000087E090EBDC018093F70154
:103A10009093F801A093F901B093FA019CE088E13A
:103A20000FB6F894A895809360000FBE9093600045
:103A3000FFCF28E0929FF0011124E80FF11DE05222
:103A4000FF4F9491892F8F7092959F700895CF9317
:103A5000C82FCB010E94191D282F30E080E1989FCC
:103A6000A0011124422B532B4038510519F480E05A
:103A700090E015C09770E92FF0E088E0C89FE00D56
:103A8000F11D112484E0EE0FFF1F8A95E1F7E20F8C
:103A9000F31FEE0FFF1FE050F84985919491CF91ED
:103AA000089580E090E0089508958091E10180FFFD
:103AB0000BC06091100185E0689FB00111247595DD
:103AC0006795759567952BC081FF09C060911001BE
:103AD00085E0689FB00111247595679520C082FF2D
:103AE00007C06091100185E0689FB001112417C0E4
:103AF0009091E2019923D1F060910F01961788F718
:103B00002091100185E0289F90011124929FA0012F
:103B1000939F500D112470E0CA010E941125603856
:103B2000710540F46115710539F002C065E070E07F
:103B3000862F08958FE7089581E008958091E1012F
:103B400080FF08C060910E0170E0759567957595CE
:103B5000679521C081FF06C060910E0170E07595E8
:103B6000679519C082FF04C060910E0170E010C01B
:103B70009091E2019923C1F060910D019617A0F791
:103B800080910E01899FC001112470E00E941125CF
:103B90006038710528F46115710521F0862F0895AC
:103BA0008FE7089581E0089561E070E0F4CF803FF1
:103BB00021F40E94551D819504C0813F29F40E9483
:103BC000551D8093E5010895823F21F40E94551D03
:103BD000819504C0833F29F40E94551D8093E40120
:103BE0000895893F19F40E949E1D05C08A3F31F453
:103BF0000E949E1D81958093E60108958B3F21F4DC
:103C00000E949E1D819504C08C3F29F40E949E1D38
:103C10008093E7010895843F21F48091E30181605E
:103C200017C0853F21F48091E301826011C0863F77
:103C300021F48091E30184600BC0873F21F48091DF
:103C4000E301886005C0883F31F48091E301806121
:103C50008093E30108958D3F21F48091E10181601B
:103C60000BC08E3F21F48091E101826005C08F3F3F
:103C700029F48091E10184608093E1010895803FFF
:103C800039F48091E50187FF6CC01092E50169C0AD
:103C9000813F29F48091E5011816BCF362C0909130
:103CA000E401823F29F497FF5CC01092E40159C0FF
:103CB000833F19F41916CCF354C0893F41F4809125
:103CC000E60118160CF04DC01092E6014AC08A3F7A
:103CD00029F48091E60187FF44C0F6CF8B3F39F489
:103CE0008091E70187FF3DC01092E7013AC08C3F09
:103CF00029F48091E7011816BCF333C0843F21F406
:103D00008091E3018E7F17C0853F21F48091E3010C
:103D10008D7F11C0863F21F48091E3018B7F0BC022
:103D2000873F21F48091E301877F05C0883F31F40C
:103D30008091E3018F7E8093E30113C08D3F21F4D6
:103D40008091E1018E7F0BC08E3F21F48091E101D3
:103D50008D7F05C08F3F29F48091E1018B7F809397
:103D6000E1018091E40181110EC08091E501811192
:103D70000AC08091E601811106C08091E70181119E
:103D800002C01092E20108958091D90183FF7EC0A4
:103D90008BE394E00E946D058091E3011F928F9365
:103DA00086E394E09F938F930E94060684E394E059
:103DB0000E946D058091E401282F082E000C330B22
:103DC0003F938F9381E394E09F938F930E94060625
:103DD0008FE294E00E946D058091E501282F082E66
:103DE000000C330B3F938F938CE294E09F938F935F
:103DF0000E9406068AE294E00E946D058091E60129
:103E0000282F082E000C330B3F938F9387E294E00A
:103E10009F938F930E94060685E294E00E946D05B1
:103E20008091E701282F082E000C330B3F938F93CE
:103E300082E294E09F938F930E9406068FE194E0C4
:103E40000E946D058091E2011F928F938CE194E0B6
:103E50009F938F930E9406068AE194E00E946D056D
:103E60008091E1011F928F9387E194E09F938F935C
:103E70000E94060684E194E00E946D058DB79EB70E
:103E80004C960FB6F8949EBF0FBE8DBF83EE91E0A7
:103E90000E94F4100E94901C9093E0018093DF0137
:103EA00008951F93CF93DF938091DF019091E001FC
:103EB0000E94A81CAC019091E201992321F020916D
:103EC000110130E006C0209112018AE0289F900184
:103ED00011244217530708F485C08091E401C09172
:103EE000E501D091E6011091E701811107C0C111F0
:103EF00075C0D11173C0111171C074C09F3F19F00A
:103F00009F5F9093E201181624F40E94551D809340
:103F1000E4018091E40187FF05C00E94551D819551
:103F20008093E4011C1624F40E94551D8093E50142
:103F30008091E50187FF05C00E94551D8195809302
:103F4000E5016091E401662331F1C091E501CC23E4
:103F500011F1062E000C770B880B990B0E940C2494
:103F600023E333E343E35FE30E9470240E94D423FE
:103F70006093E4016C2FCC0F770B880B990B0E9498
:103F80000C2423E333E343E35FE30E9470240E94A5
:103F9000D4236093E5011D1624F40E949E1D809396
:103FA000E6018091E60187FF05C00E949E1D819574
:103FB0008093E601111624F40E949E1D8093E70170
:103FC0008091E70187FF05C00E949E1D8195809327
:103FD000E701DF91CF911F910C94C41E9F3F09F020
:103FE0008FCF97CFDF91CF911F910895E3EEF1E04E
:103FF00085E0DF011D928A95E9F71092E2011092A7
:10400000E10108958EE596E00E946D051F9281E022
:104010008F931F9285E08F9380E196E09F938F931B
:104020000E9406060F900F900F900F900F900F9028
:1040300008958330E9F128F4813061F0823009F18C
:104040000895853009F462C008F449C0863009F447
:1040500074C0089580911201262F30E0280F311D81
:104060002F3F310524F4680F6093120103C08FEFD6
:1040700080931201809112011F928F9389E495E041
:1040800072C080911101262F30E0280F311D2F3F83
:10409000310524F4680F6093110103C08FEF809302
:1040A0001101809111011F928F9387E395E05BC00E
:1040B00080911001262F30E0280F311D2F3F310550
:1040C00024F4680F6093100103C08FEF80931001F8
:1040D000809110011F928F9384E295E044C08091FB
:1040E0000F01262F30E0280F311D2F3F310524F41A
:1040F000680F60930F0103C08FEF80930F018091D1
:104100000F011F928F938FE095E02DC080910E01DB
:10411000262F30E0280F311D2F3F310524F4680F82
:1041200060930E0103C08FEF80930E0180910E010A
:104130001F928F9386EF94E016C080910D01262F79
:1041400030E0280F311D2F3F310524F4680F6093B4
:104150000D0103C08FEF80930D0180910D011F921F
:104160008F938BED94E09F938F930E9406060F90A0
:104170000F900F900F900895833081F128F48130D3
:1041800059F08230D1F00895853009F449C0B8F172
:10419000863009F456C0089580911201681720F402
:1041A000861B8093120102C01092120180911201AD
:1041B0001F928F938CEC94E054C08091110168178A
:1041C00020F4861B8093110102C01092110180918E
:1041D00011011F928F938AEB94E043C080911001EC
:1041E000681720F4861B8093100102C01092100102
:1041F000809110011F928F9387EA94E032C08091E2
:104200000F01681720F4861B80930F0102C01092E3
:104210000F0180910F011F928F9382E994E021C0DA
:1042200080910E01681720F4861B80930E0102C056
:1042300010920E0180910E011F928F9389E794E0F6
:1042400010C080910D01681720F4861B80930D012A
:1042500002C010920D0180910D011F928F938EE587
:1042600094E09F938F930E9406060F900F900F90FB
:104270000F900895CF93C82F1F928F9383E697E0F6
:104280009F938F930E94060681E090E0A0E0B0E04B
:10429000BC01CD0104C0660F771F881F991FCA9506
:1042A000D2F70E941E1A0F900F900F900F90CF918F
:1042B0000C942A16CF93873288F58E3108F00BC103
:1042C0008E3009F487C0D8F4873009F460C08B3091
:1042D00009F44FC0863009F002C18091D901817F75
:1042E0008E7F8093D90188E697E00E946D058BE26E
:1042F0009AE00E946D0581E08093E90146C0863115
:1043000009F4B0C020F4803109F47AC0E8C08931E2
:1043100009F491C08B3109F449C0E1C0883349F1F7
:1043200050F4893209F4D5C0853309F4D2C08732FC
:1043300009F0D5C0CEC0833409F4CBC028F48A3349
:1043400008F4CDC08953C8C0883409F0C8C00E94A1
:104350002A168AE19AE00E946D052FEF83ED90E323
:10436000215080409040E1F700C000000E94F71CFF
:104370000CC08FE897E041C081E09AE00E946D0593
:104380008091D90181608093D901C1E0ADC0809155
:10439000D901C82FC17080FFEFCF8DE09AE00E9455
:1043A0006D058091D901817F8E7F3FC09091D901A9
:1043B00091FBCC27C0F981E0C827892FC0FB81F988
:1043C0008093D901CC2319F084EF99E029C086EEBF
:1043D00099E013C09091D90192FBCC27C0F981E0FC
:1043E000C827892FC0FB82F98093D901CC2319F00B
:1043F00087ED99E015C087EC99E00E946D05C5CF67
:104400009091D90193FBCC27C0F981E0C827892F6F
:10441000C0FB83F98093D901CC2351F08BEB99E059
:104420000E946D058091D90181608093D9015CC0A3
:104430008EEA99E0E2CF8FE999E00E946D0587E767
:1044400099E00E946D058DE299E00E946D0580E083
:1044500099E00E946D058BEB98E00E946D058DE858
:1044600098E0CBCF8FE798E00E946D050E949F10E7
:104470001F928F9385E698E09F938F930E94060684
:1044800080910A011F928F938EE498E09F938F93FF
:104490000E940606809176011F928F938BE398E02D
:1044A0009F938F930E9406060E949C1C9F938F935C
:1044B0007F936F9384E298E09F938F930E94060608
:1044C0008DB79EB742960FB6F8949EBF0FBE8DBFB4
:1044D0005CCF80E001C08D510E943A2156CF82E22C
:1044E00098E00E946D05C0E08C2FCF91089580E088
:1044F000089580E00895CF93C82F8091E90181301D
:1045000081F020F0823009F44FC046C1E0910B01E8
:10451000F0910C018081813169F0823209F03EC155
:1045200009C0E0910B01F0910C018081813111F003
:10453000823261F48C2F0E947722811104C08C2F6B
:104540000E945A212FC081E090E02CC08C2F0E9445
:104550007922811126C0C431E1F070F4CB3081F0B2
:10456000C031D1F40E9402208BE597E00E946D05D6
:1045700082E08093E90115C0C93259F0C83361F473
:1045800088E697E00E946D058FE597E00E946D0533
:1045900008C01092E90104C189E597E00E946D0509
:1045A000FFC081E08170FEC0C43228F5CE3108F032
:1045B000C1C0CB30A1F1D0F4C73009F0D3C08EE137
:1045C0008093120182E3809311018AE080931001AD
:1045D00084E180930F0188E080930E0188E280934C
:1045E0000D018FEF95E00E946D05BFC0C33149F109
:1045F000C431C1F0B7C0CB3409F4A9C028F4C93222
:1046000089F0C83361F0AEC0C13509F49EC0C2352F
:1046100009F499C0CE3409F0A5C06AE09EC00E949A
:104620000220A3C08091E801882319F01092E801CC
:104630009CC08CE096E00E946D0581E08093E901CA
:10464000B1C086EE95E00E946D0584ED95E00E9474
:104650006D05809112011F928F9381ED95E09F93DC
:104660008F930E9406068FEC95E00E946D058DEBFE
:1046700095E00E946D05809111011F928F938AEB46
:1046800095E09F938F930E94060688EB95E00E9429
:104690006D0589EA95E00E946D05809110011F92D9
:1046A0008F9386EA95E09F938F930E94060684EA93
:1046B00095E00E946D0583E995E00E946D0580916B
:1046C0000F011F928F9380E995E09F938F930E9433
:1046D00006068EE895E00E946D0589E795E00E9448
:1046E0006D0580910E011F928F9386E795E09F9351
:1046F0008F930E94060684E795E00E946D058DE584
:1047000095E00E946D0580910D011F928F938AE5BF
:1047100095E09F938F930E94060688E595E00E949E
:104720006D058DB79EB748960FB6F8949EBF0FBE25
:104730008DBF1BC0CE51EC2FF0E0E95DFE4F8081B4
:104740008093E80112C061E003C061E006C06AE046
:104750008091E8010E94192008C08091E8010E9420
:10476000BC2003C08DEF95E013C08091E801882341
:1047700069F01F928F9387EF95E09F938F930E942C
:1047800006060F900F900F900F9004C084EF95E0F5
:104790000E946D0581E006C01092E90180E002C030
:1047A00080E000CFCF9108950E94DB236894B1117F
:1047B0000C946A2408950E944F2488F09F5798F023
:1047C000B92F9927B751B0F0E1F0660F771F881F16
:1047D000991F1AF0BA95C9F714C0B13091F00E9430
:1047E0006924B1E008950C946924672F782F8827F5
:1047F000B85F39F0B93FCCF3869577956795B39557
:10480000D9F73EF490958095709561957F4F8F4FC5
:104810009F4F0895E89409C097FB3EF490958095CA
:10482000709561957F4F8F4F9F4F9923A9F0F92F76
:1048300096E9BB279395F695879577956795B795F4
:10484000F111F8CFFAF4BB0F11F460FF1BC06F5FDA
:104850007F4F8F4F9F4F16C0882311F096E911C0EC
:10486000772321F09EE8872F762F05C0662371F00D
:1048700096E8862F70E060E02AF09A95660F771F21
:10488000881FDAF7880F9695879597F9089557FD51
:104890009058440F551F59F05F3F71F04795880FAE
:1048A00097FB991F61F09F3F79F087950895121645
:1048B00013061406551FF2CF4695F1DF08C01616F1
:1048C00017061806991FF1CF8695710561050894A2
:1048D0000895E894BB2766277727CB0197F90895B9
:1048E0000E9483240C94F4240E94E62438F00E9451
:1048F000ED2420F0952311F00C94DD240C94E32496
:1049000011240C946A240E94472470F3959FC1F3EC
:10491000950F50E0551F629FF001729FBB27F00D6D
:10492000B11D639FAA27F00DB11DAA1F649F6627C2
:10493000B00DA11D661F829F2227B00DA11D621F11
:10494000739FB00DA11D621F839FA00D611D221FCB
:10495000749F3327A00D611D231F849F600D211DAF
:10496000822F762F6A2F11249F5750409AF0F1F032
:1049700088234AF0EE0FFF1FBB1F661F771F881F9B
:1049800091505040A9F79E3F510580F00C94DD24D2
:104990000C946A245F3FE4F3983ED4F386957795B0
:1049A0006795B795F795E7959F5FC1F7FE2B880F41
:1049B000911D9695879597F9089597F99F6780E8D7
:1049C00070E060E008959FEF80EC089500240A9461
:1049D0001616170618060906089500240A941216DA
:1049E0001306140605060895092E0394000C11F40D
:1049F000882352F0BB0F40F4BF2B11F460FF04C0BA
:104A00006F5F7F4F8F4F9F4F0895991B79E004C0D0
:104A1000991F961708F0961B881F7A95C9F78095FD
:104A2000089597FB072E16F4009407D077FD09D060
:104A30000E942B2507FC05D03EF4909581959F4F51
:104A40000895709561957F4F0895EE0FFF1F0590B3
:104A5000F491E02D0994AA1BBB1B51E107C0AA1FCA
:104A6000BB1FA617B70710F0A61BB70B881F991F0F
:104A70005A95A9F780959095BC01CD010895F894B9
:024A8000FFCF66
:104A82000A09FB09D809A409700901CF01280814F1
:104A92000A321E404D3622AF0362032C030A0396EC
:104AA20002AF02C802E10201020304050607080977
:024AB200000002
:106800008800EA44E944E244040005000600070069
:10681000080009000A000B000C000D000E000F001C
:1068200010001100120013001400150016001700CC
:10683000180019001A001B001C001D001E001F007C
:10684000200021002200230024002500260027002C
:10685000280029002A002B002C002D002E002F00DC
:10686000300031003200330034003500360037008C
:10687000380039003A003B003C003D003E003F003C
:1068800040004100420043004400450046004700EC
:10689000480049004A004B004C004D004E004F009C
:1068A000500051005200530054005500560057004C
:1068B000580059005A005B005C005D005E005F00FC
:1068C000600061006200630064006500850067008D
:1068D000680069006A006B006C006D006E006F005C
:1068E0007000710072007300890087008A008B00BD
:1068F000E000E100E200E300F1A1E500E600E700CE
:106900000100010001000100EA4401000100E2442D
:106910000100010001000100460001004A004B0097
:10692000010001004700480001000100E9440100A6
:106930000100010001000100010001003A003B00DC
:106940003C003D003E003F0040004100420043004B
:10695000010035004C0039000100440045005200A0
:1069600049000100010050004F0029004D004E0079
:1069700051000100680069006A006B006C006D0046
:106980006E006F0070007100720073000100010062
:1069900001000100010001000100010001004D00A3
:1069A0004A004E004B0001000100010001000100FF
:1069B00001000100010001000100010001000100CF
:1069C00001000100010001000100010001000100BF
:1069D00001000100010001000100010001000100AF
:1069E0000100010001000100490001000100010057
:1069F000010001000100010001000100010001008F
:00000001FF
